:020000040000FA
:0A00000020280000000000008828FE
:1000400003136400831681018312C0308B000130DA
:1000500083168C0083128C01831608308E00831265
:100060008312850107309F0020308316850083129C
:100070008601831686018312A101A201A301A401B6
:10008000A501A601A701A9013C30A00083169B0190
:100090001C141A088312AC0083169B0A1C141A083D
:1000A0008312AD0083169B0A1C141A088312AE003B
:1000B00009309000970183122C088F002D088E00C4
:1000C0000430A800200803190000851E6228A91426
:1000D0002008003E031D7428831686012030850009
:1000E00083123C30A0007A282808003E0319033010
:1000F000FF3EA800A9187A28A914A9187D28851AF6
:100100007F28A914A9188228A914A918852862286B
:10011000AA00030E8312AB000C102D088E072C08CA
:100120000318013E8F07A10A2108053C031DA828DA
:10013000A101A9018312A20A22082E02031DA828E8
:10014000A20028088207B828E428EB28F228FA2819
:100150002008003E0319B328210882070229072935
:100160000C29112916292B0E8300AA0E2A0E09002C
:100170002008003E0319C328A00BC3288316FF30B4
:10018000860085008312A30A23083C3C031DA8288F
:10019000A300A40A24083C3C031DA828A400A50A27
:1001A0002508183C031DA828A500A60A2608203CFF
:1001B000031DA8280130A600A70A27080D3C031D2F
:1001C000A8280130A700A828A40A24083C3C031D45
:1001D000A828A400A828A50A2508183C031DA828BB
:1001E000A500A828A60A2608203C031DA82801303F
:1001F000A600A828A70A27080D3C031DA82801303F
:10020000A700A8281E30850023088600B3281D30CB
:10021000850024088600B3281B3085002508860049
:10022000B3281730850026088600B3280F308500D4
:0602300027088600B32838
:084000000B000C00010001009F
:02400E00493F28
:06420000F900C1007D0081
:00000001FF
